:020000040000FA
:040000000FEF1AF0F4
:08000800056ED8CF06F0E0CF31
:1000100007F00001E9CF0DF0EACF08F0E1CF09F0D9
:10002000E2CF0AF0D9CF0BF0DACF0CF0F3CF14F017
:10003000F4CF15F0FACF16F000C00FF001C010F0A9
:1000400002C011F003C012F004C013F0F2AA2CEFAA
:1000500000F0F2B47FEF01F00FC000F010C001F02B
:1000600011C002F012C003F013C004F00E8E0DC0D8
:10007000E9FF08C0EAFF09C0E1FF0AC0E2FF0BC0C8
:10008000D9FF0CC0DAFF14C0F3FF15C0F4FF16C08F
:10009000FAFF055007C0E0FF06C0D8FF1000F2CFFE
:1000A0000EF0F29EF76AB80FF66E000EF722090006
:1000B000F5500EBEF28E1200008040C020A060E01D
:1000C000109050D030B070F0088848C828A868E870
:1000D000189858D838B878F8048444C424A464E440
:1000E000149454D434B474F40C8C4CCC2CAC6CEC10
:1000F0001C9C5CDC3CBC7CFC028242C222A262E210
:10010000129252D232B272F20A8A4ACA2AAA6AEA0F
:100110001A9A5ADA3ABA7AFA068646C626A666E6DF
:10012000169656D636B676F60E8E4ECE2EAE6EEEAF
:100130001E9E5EDE3EBE7EFE018141C121A161E1C7
:10014000119151D131B171F1098949C929A969E9DF
:10015000199959D939B979F9058545C525A565E5AF
:10016000159555D535B575F50D8D4DCD2DAD6DED7F
:100170001D9D5DDD3DBD7DFD038343C323A363E37F
:10018000139353D333B373F30B8B4BCB2BAB6BEB7F
:100190001B9B5BDB3BBB7BFB078747C727A767E74F
:1001A000179757D737B777F70F8F4FCF2FAF6FEF1F
:1001B0001F9F5FDF3FBF7FFF0DAE03D0F2CF0EF07A
:1001C000F29EF76ADA0FF66E010EF7220900F5507B
:1001D0000DAE02D00EBEF28E120000102030405044
:1001E00060700000000000000000F2CF0EF0F29EF0
:1001F000F76A040FF66E020EF7220900F5500EBEE4
:10020000F28E12002530344C58303030310002016B
:10021000536B546B92948994C950610EC96EC73068
:10022000FEE3C950C96AC730FEE3C950036A536F81
:1002300003C054F253C203F0000E536F03C054F2D4
:10024000C950C96AC730FEE3C95053135431036E15
:100250005331026E033202323F0E031602C053F2D4
:1002600003C054F2000B006E5451200B036E00507B
:10027000031002E0C00E541353C201F054C202F046
:10028000000144EF01F0C3D702C052F201C051F2A5
:10029000020151C201F052C202F00001000C92941E
:1002A00089940201535180095411566FC95056C2A6
:1002B000C9FFC730FEE3929489840001000C02015B
:1002C0004F51020802E14F6B09D04F5303E1010E79
:1002D0004F6F04D04F2D02D0020E4F6F036A505162
:1002E000F2CF51F2F29E000167DF020151BFF28EA0
:1002F000526F4FC253F2546F0001D1DF000CEC512A
:10030000EA2502014F6F0001ED51EB210201D76E8A
:100310004FC2D6FF0001EE2BD8B4EF2BED6BEC6B88
:10032000EF5303E1EE51020805E2EF6BEE6BED6B6C
:10033000140EEC6FDF2BE851DF5D15E1E95313E19B
:10034000DF6BDE2BDE510A080EE1DE6BDD2BDD51AB
:100350003C0809E1DD6BDC2BDC513C0804E1DC6B83
:10036000DA2BD8B4DB2B0101E62D91D0E75327E13E
:10037000D890E035026EE135036E0250F00F016E49
:10038000000E032201C04FF203C050F200017BDFD8
:1003900050C2EAFF4FC2E9FF02C0ECFFED5201C0BC
:1003A000EFFF010E0101E76F02014F6FE8C150F24C
:1003B000000185DF0101E02BD8B4E12B51D0E72DFE
:1003C00027D0D890E035026EE135036E0250F00F71
:1003D000016E000E032201C04FF203C050F2000173
:1003E00052DF50C2EAFF4FC2E9FF02C0ECFFED52FC
:1003F00001C0EFFF020E0101E76F02014F6FE9C17B
:1004000050F200015CDF0101E02BD8B4E12B28D0D1
:10041000E751020825E1D890E035026EE135036E20
:100420000250F00F016E000E032201C04FF203C014
:1004300050F2000128DF50C2EAFF4FC2E9FF02C0BC
:10044000ECFFED5201C0EFFF0101E76B02014F6BC2
:10045000E8C150F2000133DF0101E02BD8B4E12BF9
:10046000E0513C0808E1E15306E1E56BE46BE36B26
:10047000010EE26F0CD0E051780809E1E15307E189
:10048000E56BE46BE36B020EE26FE16BE06BF29401
:1004900000012CEF00F0010EEA6EFC0EE96EEF5049
:1004A0000EE00C0E016E006A002EFED7012EFBD767
:1004B000F70E006E002EFED700D0EF2EF2D7000C04
:1004C000EBC0D7FFEAC0D6FF0101FCC1E9FFFDC1C7
:1004D000EAFFEC6AED52EF6A020EFC25E96E000EAF
:1004E000FD21EA6EEF6A030EFC25E96E000EFD2188
:1004F000EA6EEF6A040EFC25E96E000EFD21EA6E3D
:10050000EF6A050EFC25E96E000EFD21EA6EEF6A2A
:100510000001000C92948994C950180EC96EC7301E
:10052000FEE3C950C96AC730FEE392948984AEEFF6
:1005300002F0929489940101FAC1FCF1C950FAC108
:10054000C9FFC730FEE3C950FBC1C9FFC730FEE396
:10055000929489840001B5EF02F0DCD7070E010107
:10056000FA6F3E0EFB6F0001E4D792908990F1EF95
:100570000EF0016A026A006A036A02010A5102E18E
:10058000095118E0100E0B6FD89007370837003666
:1005900003360A51035C02E10951005C07E309518B
:1005A000005ED8A003060A51035ED88001360236E9
:1005B0000B2FEAD700014FEF0DF08E0E006E2BC20D
:1005C00001F02AC202F0036A015209E102C001F0FF
:1005D000026A080E005E015202E1006A08D0D8905B
:1005E00001BE04D0023601360006F9D7019E000C88
:1005F0003BC242F202013F51421B42AF05D0D894A8
:10060000D8903BBFD8802FD03BC242F23EC243F2CB
:100610003A51435F06E042AF26D0D850010AD86E67
:1006200022D03FC243F23B51435F06E042AF1BD0B2
:10063000D850010AD86E17D040C243F23C51435FF4
:1006400006E042AF10D0D850010AD86E0CD041C29B
:1006500043F23D51435F06E042AF05D0D850010A56
:10066000D86E01D0D8900001000C800ED8A202D024
:100670000201431B0201486B496B3FC247F24351E1
:10068000471B3E51D8B4DFD0466F006E4251D8B4FC
:10069000E3D0465FD8B483D03EE343C24CF24C8FE4
:1006A00044C24BF245C24AF2496BD8904C334B33AB
:1006B0004A334933462FF8D747AF03D04881E0D0BB
:1006C000489146914889020EEA6E410EE96EEBD0E0
:1006D000489947BF0AD046A113D04C334B334A3315
:1006E0004933002AD8B4C7D00BD04CBF0CD0D89017
:1006F00049374A374B374C370006D8B4BCD0F5D70A
:10070000488D6DD0489D3FC247F23FAF02D04C8F1D
:10071000ABD04C9FA9D042C246F242C200F03E513B
:10072000465F3FC24CF24C8F40C24BF241C24AF28C
:10073000496BD8904C334B334A334933462FF8D763
:1007400047AF03D048839CD048934691488B020E14
:10075000EA6E450EE96EA7D0489B47BF0AD046A176
:1007600013D04C334B334A334933002AD8B483D0A7
:100770000BD04CBF0CD0D89049374A374B374C3749
:100780000006D8B478D0F5D7488F29D0489F43C207
:1007900047F243AF02D04C8F67D04C9F65D043C225
:1007A0004CF24C8F44C24BF245C24AF247AF04D0E0
:1007B0004C9F488565D04895496B4691020EEA6E7C
:1007C000410EE96E70D047BF1CD03FC247F246A130
:1007D00006D04C334B334A334933002A4CE049AFFF
:1007E0000BD04A2B09E14B2B07E14C2B05E14C3395
:1007F0004B334A33002A3FE048BD84D748BFC6D7B1
:100800001CD0800E4C1B4CAF04D03AD043C247F2F0
:100810000AD03FC247F24C5306E14B5304E14A531E
:1008200002E1006A21D04CBF08D0D89049374A373E
:100830004B374C37002EF7D71ED047AF02D04C8F26
:1008400013D04C9F11D042C200F043C24CF244C2BC
:100850004BF245C24AF208D03EC200F03FC24CF211
:1008600040C24BF241C24AF24CC201F04BC202F00C
:100870004AC203F034D0006A016A026A036A2FD0C8
:10088000496B4A1F4B1F4C1F491F492B05E14A2B3F
:1008900003E14B2B01E14C2B48B112D748B354D79D
:1008A00048B589D7B3D7EF504A2705E34B2B03E16F
:1008B0004C2BD8B44681ED52EF504B2703E34C2B21
:1008C000D8B44681ED52EF50EFBE01D0800A4C27DC
:1008D000D8B0468148B9FCD648BB3ED774D7000192
:1008E000000C02013E51D8B4A5D04A6F4251D8B491
:1008F000A1D04A5F05E37F0E4A27D8B09BD006D02F
:10090000810E4A5FD8A096D0D8B494D04AC200F0E5
:10091000016A026A036A496B3FC248F2488F40C2CB
:1009200047F241C246F2190E4A6F4551465F0DE249
:10093000010E475F0AE2485F08E2495F06E2492B81
:10094000482B472B4551462728D04451475F12E298
:10095000010E485F0FE2495F0DE2492B482B4451DD
:1009600047274551462719E3472B17E1482B15E147
:10097000492B13D043518009485F0EE2010E495FB5
:100980000BE2492B43518009482744514727E9E3AB
:10099000482BE7E1492BE5D703804A2F01D00BD044
:1009A000D8904637473748374937D890033602360C
:1009B00001364B37BAD74BA106D0D890013202325C
:1009C00003324B3302D0000635E04BBF1ED0D89027
:1009D00046374737483749374551465F07E2010EEA
:1009E000475F04E2485F02E2495F1AE34451475F10
:1009F00005E2010E485F02E2495F12E343518009BC
:100A0000485F03E2010E495F0BE3032A09E1022A72
:100A100007E1012A05E1002A0DE00132023203322A
:100A20003FC24AF243514A1B4AAF02D0018E06D060
:100A3000019E04D0006A016A026A036A0001000C88
:100A400002013A51D8B471D0006E3E51D8B46DD085
:100A5000002604E3810E002668E204D07F0E005ECB
:100A600064E363E03BC242F23F51421B3B8F3F8F46
:100A70003D514103F4CF44F23C514003F4CF03F025
:100A8000F3CF43F24103F3504427F4504323000EC5
:100A900003223D514003F3504427F4504323000EFA
:100AA000026A032202223B514103F3504327F450D0
:100AB0000322000E02223B514003F3500326F45060
:100AC0000222000E016A01223D513F03F3504327E9
:100AD000F4500322000E022201223C513F03F35046
:100AE0000326F4500222000E01223B513F03F35033
:100AF0000226F4500122002A01BE05D043370336F6
:100B0000023601360006000E43AF0AD0032A022245
:100B10000122015005E1025003E1035001E1002AE6
:100B200042BF018E42AF019E04D0006A016A026A90
:100B3000036A0001000C8E0E006E3DC201F03CC243
:100B400002F0036A01AE05D0011E021E022A01E175
:100B5000012A015209E102C001F0026A080E005E9A
:100B6000015202E1006A0DD0D89001BE04D00236D5
:100B700001360006F9D702013DAF02D0000101D0D5
:100B8000019E0001000C28C22CF227C22BF226C2C3
:100B90002AF225C229F22CC23DF22BC23CF22AC213
:100BA0003BF229C23AF20201416B406B3F6B7F0E70
:100BB0003E6F00011DDDD8B435D2020E02013B6F3D
:100BC000290EE96E3BC2EAFF7E0EEF6ED8822CC280
:100BD00041F22BC240F22AC23FF229C23EF2456BDB
:100BE000446B436B7F0E426F00013FDD00C03AF261
:100BF00001C03BF202C03CF203C03DF2D8922CC2CD
:100C000041F22BC240F22AC23FF229C23EF2020157
:100C1000456B446B436B7F0E426F000126DD3DC286
:100C200041F23CC240F23BC23FF23AC23EF203C044
:100C300045F202C044F201C043F200C042F251DE6C
:100C400003C02CF202C02BF201C02AF200C029F22C
:100C50002CC23DF22BC23CF22AC23BF229C23AF22C
:100C60002CC241F22BC240F22AC23FF229C23EF20C
:100C7000E7DE03C038F202C037F201C036F200C02E
:100C800035F2BC0E02013D6F240E3C6F670E3B6FC8
:100C90007D0E3A6F38C241F237C240F236C23FF29F
:100CA00035C23EF20001CCDE00C03AF201C03BF298
:100CB00002C03CF203C03DF2D89203C041F202C030
:100CC00040F201C03FF200C03EF2E30E0201456F68
:100CD000E40E446F900E436F820E426F0001C5DC3C
:100CE00003C030F202C02FF201C02EF200C02DF27C
:100CF00030C23DF22FC23CF22EC23BF22DC23AF27C
:100D000038C241F237C240F236C23FF235C23EF23B
:100D100097DE00C03AF201C03BF202C03CF203C0D1
:100D20003DF2D89203C041F202C040F201C03FF24E
:100D300000C03EF21C0E0201456F870E446F570E35
:100D4000436F830E426F000190DC03C030F202C09B
:100D50002FF201C02EF200C02DF230C23DF22FC2A0
:100D60003CF22EC23BF22DC23AF238C241F237C2F7
:100D700040F236C23FF235C23EF262DE00C03AF2C5
:100D800001C03BF202C03CF203C03DF2D89203C066
:100D900041F202C040F201C03FF200C03EF2AB0E91
:100DA0000201456FE10E446F9E0E436F830E426F4A
:100DB00000015BDC03C030F202C02FF201C02EF252
:100DC00000C02DF202013D6B3C6B3B6B7F0E3A6F16
:100DD00038C241F237C240F236C23FF235C23EF26B
:100DE00000012EDE00C03AF201C03BF202C03CF22C
:100DF00003C03DF2D89203C041F202C040F201C0EC
:100E00003FF200C03EF2B40E0201456F2A0E446F5D
:100E1000820E436F426F000128DC03C034F202C02F
:100E200033F201C032F200C031F234C23DF233C2BB
:100E30003CF232C23BF231C23AF238C241F237C21E
:100E400040F236C23FF235C23EF2FADD00C03AF25D
:100E500001C03BF202C03CF203C03DF2D89203C095
:100E600041F202C040F201C03FF200C03EF2800EEB
:100E70000201456F3E0E446F060E436F830E426FB4
:100E8000000135EC03F003C034F202C033F201C0BC
:100E900032F200C031F234C23DF233C23CF232C20F
:100EA0003BF231C23AF238C241F237C240F236C2A6
:100EB0003FF235C23EF2C4DD00C03AF201C03BF25F
:100EC00002C03CF203C03DF2D89203C041F202C01E
:100ED00040F201C03FF200C03EF2AB0E0201456F8E
:100EE000E10E446F9E0E436F820E426F000135EC9F
:100EF00003F003C034F202C033F201C032F200C08A
:100F000031F22CC23DF22BC23CF22AC23BF229C282
:100F10003AF230C241F22FC240F22EC23FF22DC24D
:100F20003EF28EDD00C03AF201C03BF202C03CF25C
:100F300003C03DF203C041F202C040F201C03FF2E3
:100F400000C03EF234C245F233C244F232C243F230
:100F500031C242F2C6DC03C030F202C02FF201C03F
:100F60002EF200C02DF2020E02013B6F250EE96E3B
:100F70003BC2EAFF7E0EEF5C396F39BF01D014D05F
:100F8000000ED88039553D6B3C6F3CBF3D070001DA
:100F9000D2DD00C031F20150800A0201326F02C07E
:100FA00033F203C034F210D03D6B39C23CF23CBF87
:100FB0003D070001C0DD03C034F202C033F201C0BE
:100FC00032F200C031F2020134C23DF233C23CF2CF
:100FD00032C23BF231C23AF2180E416F720E406FCC
:100FE000310E3F6F7E0E3E6F00012ADDD89230C277
:100FF00041F22FC240F22EC23FF22DC23EF203C098
:1010000045F202C044F201C043F200C042F235ECA6
:1010100003F003C030F202C02FF201C02EF200C074
:101020002DF206D00201306B2F6B2E6B2D6B000161
:101030002DC200F02EC201F02FC202F030C203F028
:10104000000C0EC228F20DC227F20CC226F20BC20F
:1010500025F299DD03C012F202C011F201C010F2B4
:1010600000C00FF212C241F211C240F210C23FF2B0
:101070000FC23EF28E0E0201456F5D0E446F130EDD
:10108000436F800E426F00012CDC03C012F202C0DD
:1010900011F201C010F200C00FF20FC200F010C236
:1010A00001F011C202F012C203F068EF0DF08E0ED3
:1010B000006E02013851005E39C202F03AC201F0FE
:1010C000028E005209E0D890025202E1015204E07F
:1010D00002320132002EF7D739AF05D0011E021EB1
:1010E000012AD8B4022A0001000C0201259119C27C
:1010F0001EF218C21DF217C21CF216C21BF219C250
:101100003DF218C23CF217C23BF216C23AF2416BF2
:10111000406B3F6B3E6B0001F8EC02F005E302010F
:1011200025811C51800A1C6F1EC23DF21DC23CF27B
:101130001CC23BF21BC23AF20201416B406B3F6B97
:101140008E0E3E6F0001F8EC02F001E218E11EC2C3
:101150003BF21DC23AF21CC239F21BC238F2A7DFC1
:1011600002C02BF201C02AF2DDEC02F003C022F231
:1011700002C021F201C020F200C01FF2D1D01EC275
:101180003DF21DC23CF21CC23BF21BC23AF2800E81
:101190000201416F960E406F180E3F6F960E3E6F24
:1011A0000001F8EC02F0D8A0B3D01EC241F21DC27B
:1011B00040F21CC23FF21BC23EF20201456B446B7F
:1011C000436B8E0E426F000171EC04F003C03BF2E2
:1011D00002C03AF201C039F200C038F268DF02C042
:1011E00024F201C023F21EC241F21DC240F21CC211
:1011F0003FF21BC23EF20201456B446B436B8E0E05
:10120000426F000171EC04F000C026F201C027F229
:1012100002C028F203C029F224C22BF223C22AF210
:10122000DDEC02F0D88229C241F228C240F227C286
:101230003FF226C23EF203C045F202C044F201C0B2
:1012400043F200C042F235EC03F002013D6B3C6B0F
:101250003B6B8E0E3A6F03C041F202C040F201C0F8
:101260003FF200C03EF2000120EC05F003C01EF288
:1012700002C01DF201C01CF200C01BF224C22BF2FE
:1012800023C22AF2DDEC02F002013D6B3C6B3B6BAA
:101290008E0E3A6F03C041F202C040F201C03FF22D
:1012A00000C03EF2000120EC05F003C022F202C0B3
:1012B00021F201C020F200C01FF21EC23BF21DC28B
:1012C0003AF21CC239F21BC238F2F1DE02C02BF234
:1012D00001C02AF2DDEC02F0D89222C241F221C212
:1012E00040F220C23FF21FC23EF203C045F202C0EC
:1012F00044F201C043F200C042F235EC03F003C0F7
:1013000022F202C021F201C020F200C01FF208D078
:101310001EC222F21DC221F21CC220F21BC21FF209
:101320001EC23BF21DC23AF21CC239F21BC238F295
:10133000BEDE02C02BF201C02AF2DDEC02F0D88240
:101340001EC241F21DC240F21CC23FF21BC23EF25D
:1013500003C045F202C044F201C043F200C042F2B1
:1013600035EC03F003C01EF202C01DF201C01CF2F6
:1013700000C01BF2020125A103D02051800A206F7A
:101380001EC23DF21DC23CF21CC23BF21BC23AF22D
:10139000416B406B3F6B3E6B0001F8EC02F03CE0B0
:1013A000020125A11CD01A531AE1D88222C241F2AF
:1013B00021C240F220C23FF21FC23EF2456B446B95
:1013C000436B7F0E426F000135EC03F003C022F245
:1013D00002C021F201C020F200C01FF2020125B1BB
:1013E0001CD01A2D1AD0D89222C241F221C240F24A
:1013F00020C23FF21FC23EF2456B446B436B7F0E2F
:10140000426F000135EC03F003C022F202C021F26A
:1014100001C020F200C01FF2020119C23DF218C241
:101420003CF217C23BF216C23AF2416B406B3F6B83
:101430003E6B0001F8EC02F006E10201226B216B29
:10144000206B1F6B00011FC200F020C201F021C2FF
:1014500002F022C203F039EF0AF015C219F214C2E9
:1014600018F213C217F212C216F202011A6B00012F
:101470003CD6000C29C241F228C240F227C23FF2FA
:1014800026C23EF2180E0201456F720E446F310EF5
:10149000436F7E0E426F000171EC04F003C03BF21B
:1014A00002C03AF201C039F200C038F200DE01C0D9
:1014B00036F20201379129C22DF228C22CF227C23E
:1014C0002BF226C22AF229C23DF228C23CF227C2E0
:1014D0003BF226C23AF2416B406B3F6B3E6B000120
:1014E000F8EC02F006E302013781366D2B51800AD9
:1014F0002B6F0201316B306B2F6B2E6B020E396F2D
:101500002E0EE96E39C2EAFF7F0E3625EF6E2DC230
:1015100041F22CC240F22BC23FF22AC23EF2180E18
:10152000456F720E446F310E436F7E0E426F0001A5
:1015300071EC04F000C038F201C039F202C03AF296
:1015400003C03BF202013D6B36C23CF23CBF3D079B
:1015500000019BEC05F0D8823BC241F23AC240F256
:1015600039C23FF238C23EF203C045F202C044F233
:1015700001C043F200C042F235EC03F003C02DF28B
:1015800002C02CF201C02BF200C02AF27C0E020134
:101590003D6F880E3C6F590E3B6F720E3A6F2DC235
:1015A00041F22CC240F22BC23FF22AC23EF20001AD
:1015B00020EC05F000C038F201C039F202C03AF266
:1015C00003C03BF2D89203C041F202C040F201C016
:1015D0003FF200C03EF2E00E0201456F970E446FED
:1015E000260E436F750E426F000135EC03F003C009
:1015F00035F202C034F201C033F200C032F235C21B
:101600003DF234C23CF233C23BF232C23AF22DC256
:1016100041F22CC240F22BC23FF22AC23EF220EC31
:1016200005F000C038F201C039F202C03AF203C03E
:101630003BF2D89203C041F202C040F201C03FF237
:1016400000C03EF2C40E0201456F1D0E446F1E0E17
:10165000436F780E426F000135EC03F003C035F2A2
:1016600002C034F201C033F200C032F235C23DF2A2
:1016700034C23CF233C23BF232C23AF22DC241F2E2
:101680002CC240F22BC23FF22AC23EF220EC05F0FF
:1016900000C038F201C039F202C03AF203C03BF296
:1016A000D89203C041F202C040F201C03FF200C034
:1016B0003EF25E0E0201456F500E446F630E436FA3
:1016C0007A0E426F000135EC03F003C035F202C020
:1016D00034F201C033F200C032F235C23DF234C2FE
:1016E0003CF233C23BF232C23AF22DC241F22CC27A
:1016F00040F22BC23FF22AC23EF220EC05F000C0BD
:1017000038F201C039F202C03AF203C03BF2D8927B
:1017100003C041F202C040F201C03FF200C03EF2FD
:101720001A0E0201456FFE0E446F750E436F7C0E5C
:10173000426F000135EC03F003C035F202C034F211
:1017400001C033F200C032F235C23DF234C23CF285
:1017500033C23BF232C23AF22DC241F22CC240F205
:101760002BC23FF22AC23EF220EC05F000C038F254
:1017700001C039F202C03AF203C03BF2D89203C072
:1017800041F202C040F201C03FF200C03EF2180E2A
:101790000201456F720E446F310E436F7E0E426F31
:1017A000000135EC03F003C035F202C034F201C091
:1017B00033F200C032F22DC23DF22CC23CF22BC2F9
:1017C0003BF22AC23AF235C241F234C240F233C28D
:1017D0003FF232C23EF220EC05F0D8920201416B9A
:1017E000406B3F6B7F0E3E6F03C045F202C044F278
:1017F00001C043F200C042F2000135EC03F031C2F7
:101800003DF230C23CF22FC23BF22EC23AF203C08C
:1018100041F202C040F201C03FF200C03EF220ECB3
:1018200005F003C031F202C030F201C02FF200C057
:101830002EF2020137A119D0416B406B3F6B7F0E36
:101840003E6F31C245F230C244F22FC243F22EC283
:1018500042F2000171EC04F003C031F202C030F238
:1018600001C02FF200C02EF202012EC200F02FC2E2
:1018700001F030C202F031C203F00001000C02019D
:101880003D6B3C6B3B6B3A6B1CC241F21BC240F29E
:101890001AC23FF219C23EF20001F8EC02F001E276
:1018A0002FE11CC228F21BC227F21AC226F219C26B
:1018B00025F2C3EC05F020C23DF21FC23CF21EC26D
:1018C0003BF21DC23AF203C041F202C040F201C035
:1018D0003FF200C03EF220EC05F000C021F201C052
:1018E00022F202C023F203C024F203C029F202C094
:1018F00028F201C027F200C026F2BCDD3BD03AD06E
:1019000019C221F202011A51800A226F1BC223F26E
:101910001CC224F21CC228F21BC227F2266F19C275
:1019200025F20001C3EC05F020C23DF21FC23CF2DB
:101930001EC23BF21DC23AF203C041F202C040F2A5
:1019400001C03FF200C03EF220EC05F000C022F2E0
:1019500001C023F202C024F203C025F203C029F221
:1019600002C028F201C027F200C026F283DD800EFB
:10197000011A00D0E3EF0CF0800E0201116F126B20
:10198000136B146B3D6B10C23CF23CBF3D07000172
:101990009BEC05F000C015F201C016F202C017F270
:1019A00003C018F214C21CF213C21BF212C21AF2C4
:1019B00011C219F203C020F202C01FF201C01EF2D0
:1019C00000C01DF25CD70FC23DF20EC23CF20DC248
:1019D0003BF20CC23AF203C041F202C040F201C035
:1019E0003FF200C03EF220EC05F0B4EF0DF0080E1F
:1019F000016E0A0E006E0400002EFDD78B909490AD
:101A00000A0E006E0400002EFDD702010A378B92E9
:101A1000D8B09482D8A09492948082A0FED7012E50
:101A200001D002D00001E5D70A0E006E0400002E9E
:101A3000FDD78B909490000094820A0E006E0400F3
:101A4000002EFDD70A0E006E0400002EFDD79480F4
:101A500082A0FED7016A0A0E006E0400002EFDD798
:101A600082B201808B9094908B9294920001000C32
:101A700002010151040808E303E100510E0804E3E8
:101A8000040E016F0F0E006F01C208F200C207F2D0
:101A9000040E0A6F0F0E096F0001B9EF02F002C0C9
:101AA0002BF201C02AF20001DDEC02F000C006F2C8
:101AB00001C007F202C008F203C009F203C00EF22F
:101AC00002C00DF201C00CF200C00BF221EF08F0D1
:101AD000A60E02013D6F9B0E3C6F540E3B6F800EB5
:101AE0003A6F03C041F202C040F201C03FF200C0B1
:101AF0003EF2000120EC05F000C007F201C008F240
:101B000002C009F203C00AF203C015F202C014F2C7
:101B100001C013F200C012F2A0DC03C03BF202C00D
:101B20003AF201C039F200C038F257EC08F001C0B7
:101B300003F2020103510F0802E20F0E036F8A0E37
:101B4000066F010E076FE00E086F096B0A0E032582
:101B50000A6F09C20FF208C20EF207C20DF206C2E6
:101B60000CF2106F000108D700C007F201C008F2A4
:101B700002C009F203C00AF201C22BF200C22AF22B
:101B8000DDEC02F00AC241F209C240F208C23FF2A3
:101B900007C23EF203C045F202C044F201C043F264
:101BA00000C042F271EC04F0EACF0CF2E9CF0BF284
:101BB000D8820201416B406B3F6B8A0E3E6F03C0BF
:101BC00045F202C044F201C043F200C042F20001FB
:101BD00035EC03F00CC2EAFF0BC2E9FF00C00DF2C6
:101BE00001C00EF202C00FF203C010F203C015F2E2
:101BF00002C014F201C013F200C012F22EDC03C0C6
:101C00003BF202C03AF201C039F200C038F257ECA0
:101C100008F002C005F201C004F20201033BF00E1D
:101C200003170437053704370537FC0E0417020E77
:101C3000076F040E066F010E0625016E000E0721C8
:101C400001C0E9FFEA6EEF500311EF6E020E036E62
:101C5000040EE96E03C0EAFFEF50FC0B006E036A4E
:101C60000050ED52EF6E03C0ECFF020E036E040E47
:101C7000E96E03C0EAFFEF500211006EECCF03F0F3
:101C80000050ED52EF6E03C0ECFF94820A0E006E1E
:101C90000400002EFDD794800A0E006E0400002E72
:101CA000FDD78B9294920A0E006E0400002EFDD791
:101CB0008B9094900101FF51FE0B0201066F0A6F99
:101CC000000195DE020E0201076F040E066F010E81
:101CD0000625016E000E0721036E01C0E9FFEA6EC2
:101CE000EFCF08F208C20AF2000181DE020E036E95
:101CF000040EE96E03C0EAFFECCF07F2ED52EFCF1E
:101D000006F206C20AF273DE94920000948082A06A
:101D1000FED70A0E006E0400002EFDD700D0000092
:101D200094820A0E006E0400002EFDD7000C010103
:101D3000FC5102080CE12E0EFF6FFEC101F2FDC145
:101D400000F20201026B000193DE0BD001012C0EA8
:101D5000FF6FFEC101F2FDC100F20201026B000142
:101D600087DE000CD96BD791000CB0989484BD6AC3
:101D7000796A9482BA6A676AC150C00B0F09C16E52
:101D8000C290929A899A020E0101FA6FFA0EFC6FC4
:101D900000014BEC02F00101FA2FF8D7010EEF6FB2
:101DA000900EEE6F0001E96B780EE86FFB0EEB6FA3
:101DB000EE0EEA6FED6BEC6BEF6BEE6B820ED56E99
:101DC0000101FD6BDA0EFC6F000160EC02F0C69AB7
:101DD000949A94889496210EC66E000EC76EADEF4D
:101DE00002F00101E86BE96B090EEB6FC40EEA6FBC
:101DF000270EED6F100EEC6F186AF2BE188EF29E71
:101E000002014F6BE8C150F200015FEC01F018BE17
:101E1000F28E0101E76BFC6BEBC1FEF1EAC1FDF153
:101E2000000185DF020E0101FC6FEDC1FEF1ECC186
:101E3000FDF100017CDF96DF96928D8296908D8079
:101E40000101E66BE56BE46BE36BE26BE16BE06B6E
:101E5000F36B010EF26FF16BF06FC00EF2129298FD
:101E6000899898948F84F46B000130EF1AF0010187
:101E7000FF6B988286B218D096928D92060E006EF5
:101E8000002EFED70000FF0E956E8350F2CF01F2B8
:101E9000F29E00014FEC00F0020101BFF28EE8CF8C
:101EA000FFF196928D820101FFC101F000012EEF3A
:101EB00010F00201086B096B0A6B0B6B076B065184
:101EC000075D5EE2083709370A370B3708370937ED
:101ED0000A370B37083709370A370B3708370937FE
:101EE0000A370B37F00E0817036A07510425E96E0D
:101EF00005510320EA6EEF50390820E3036A0751C9
:101F00000425E96E05510320EA6EEF5008250C6F99
:101F1000000E09210D6F000E0A210E6F000E0B211D
:101F20000F6F300E0C5D086F000E0D59096F000E1B
:101F30000E590A6F000E0F590B6F20D00A0E08259C
:101F40000C6F000E09210D6F000E0A210E6F000E9E
:101F50000B210F6F036A07510425E96E0551032019
:101F6000EA6E410EEF5C0C25086F000E0D21096F23
:101F7000000E0E210A6F000E0F210B6F072B9FD74B
:101F800008C200F009C201F00AC202F00BC203F05D
:101F90000001000C0101FD6BFE6B1B50020803E009
:101FA000000E016E43D0010E0001D85D036A1B0FC5
:101FB000E96E000E0320EA6EEF50030804E0000E05
:101FC000016E010133D0010E0101FF6F030E00010C
:101FD000D85D0101FF5D0BE2036AFF511B0FE96E43
:101FE000000E0320EA6EEF50FD27FF2BEFD7FD1FF9
:101FF000030E0001D85D036A1B0F0201026F000E81
:102000000320036F056F02C204F2020E066F000187
:1020100050DF00C0FEF10101FD51FE5D04E0000E45
:10202000016E04D003D0010E016E00D0000150EF0C
:1020300010F098DE0101FC6BFC513F0827E3988209
:1020400086B221D0036AFC511B0F016E000E0322E1
:1020500001C0FDF103C0FEF1000109D7FEC1EAFF96
:10206000FDC1E9FF01C0EFFF036A0101FC511B0F35
:10207000E96E000E0320EA6EEF50030803E1FCC195
:10208000D9F004D001D002D0FC2BD6D70001D95111
:102090003F080CE3D7B109D0010ED925D86F7AD704
:1020A000015202E0D78101D05DDE01D05BDE39EF65
:1020B0001AF0F6C1EAFFF5C1E9FF020103C2EFFF22
:1020C000E92AD8B4EA2AEF6A0101F52BD8B4F62B35
:1020D0000001000C020102BF11D00F0E006E013989
:1020E00000160A0E005C03E2300E002602D00251F8
:1020F000002600C003F20001DCDF02010F0E011711
:102100000A0E015D02E2300E02D0029F0251012749
:1021100001C203F20001CDDF000C0101FF6BFF5192
:1021200077080BE3036AFF515B0FE96E000E032093
:10213000EA6EFF0EEF6EFF2BF2D7FCC100F0FD51EF
:10214000036E05E100520001D8B4DAD0010103505A
:1021500006E1010E005C0001D8B4E3D00101035098
:1021600006E1020E005C0001D8B4EDD0010103507D
:1021700006E1030E005C0001D8B4F7D00101035062
:1021800006E1040E005C0001D8B401D10101035046
:1021900006E1050E005C0001D8B412D10101035024
:1021A00006E1060E005C0001D8B4AED10101035077
:1021B00006E1070E005C0001D8B4BFD10101035055
:1021C00006E1080E005C0001D8B4C9D1010103503A
:1021D00006E1090E005C0001D8B4E5D1010103500D
:1021E00006E10A0E005C0001D8B4FDD101010350E4
:1021F00006E10B0E005C0001D8B415D201010350BA
:1022000006E1640E005C0001D8B42CD20101800EFE
:10221000035C05E100520001D8B436D2010103503D
:1022200006E1650E005C0001D8B440D20101035004
:1022300006E1660E005C0001D8B44AD201010350E9
:1022400006E1670E005C0001D8B463D201010350BF
:1022500006E1680E005C0001D8B46ED201010350A3
:1022600006E1690E005C0001D8B480D20101035080
:1022700006E16A0E005C0001D8B48BD20101035064
:1022800006E16B0E005C0001D8B4A4D2010103503A
:1022900006E16C0E005C0001D8B4AFD2010103501E
:1022A00006E16D0E005C0001D8B4C1D201010350FB
:1022B00006E16E0E005C0001D8B4CCD201010350DF
:1022C00006E16F0E005C0001D8B4DED201010350BC
:1022D00006E1700E005C0001D8B4E9D201010350A0
:1022E00006E1710E005C0001D8B4F4D20101035084
:1022F00006E1720E005C0001D8B409D301012BD3B2
:102300000101F66B5B0EF56F0201016B370E026F78
:102310000001E0DE0201016B370E026F0001DADE20
:102320002DD30101F66B5B0EF56F0201016B370EC9
:10233000026F0001CFDE010E0201016F370E026F46
:102340000001C8DE1BD30101F66B5B0EF56F0201C5
:10235000016B370E026F0001BDDE020E0201016F3C
:10236000370E026F0001B6DE09D30101F66B5B0E7A
:10237000F56F0201016B370E026F0001ABDE030E39
:102380000201016F370E026F0001A4DEF7D20101D6
:10239000F66B5B0EF56F0201016B370E026F0001E9
:1023A00099DE040E0201016F370E026F000192DE0A
:1023B000FEC101F2370E0201026F00018BDEDED298
:1023C0000101F66B5B0EF56F0201016B370E026FB8
:1023D000000180DE050E0201016F370E026F000161
:1023E00079DE0101F66B5F0EF56FE7C001F2370E83
:1023F0000201026F00016EDEE6C001F2370E02013B
:10240000026F000167DEE5C001F2370E0201026FC4
:10241000000160DEE3C001F2370E0201026F00012D
:1024200059DEE2C001F2370E0201026F000152DEF6
:10243000E1C001F2370E0201026F00014BDE010123
:10244000F66B6B0EF56FEBC101F2370E0201026FF6
:10245000000140DEEAC101F2370E0201026F000105
:1024600039DEE8C101F2370E0201026F000132DEEF
:10247000EDC101F2370E0201026F00012BDEECC14B
:1024800001F2370E0201026F000124DEE9C101F200
:10249000370E0201026F00011DDEEFC101F2370E9F
:1024A0000201026F000116DEEEC101F2370E0201D9
:1024B000026F00010FDE0E0E0201016F370E026F78
:1024C000000108DE0101F66B7D0EF56F010E0201C1
:1024D000016F370E026F0001FDDD0201016B370E47
:1024E000026F0001F7DD020E0201006F300E036F74
:1024F0000001DFDD0201002FF9D7080E016F370E52
:10250000026F0001E7DD3AD20101F66B5B0EF56F59
:102510000201016B370E026F0001DCDD060E0201C5
:10252000016F370E026F0001D5DDFEC101F2370EDB
:102530000201026F0001CEDD21D20101F66B5B0EBC
:10254000F56F0201016B370E026F0001C3DD070E4C
:102550000201016F370E026F0001BCDD0FD20101D5
:10256000F66B5B0EF56F0201016B370E026F000117
:10257000B1DD080E0201016F370E026F0001AADD06
:10258000050E0201006F00510001F5EC00F00201A0
:10259000002B006E036F00018CDD090E0201005D4F
:1025A000F2E10001EBD10101F66B5B0EF56F020168
:1025B000016B370E026F00018DDD090E0201016F04
:1025C000370E026F000186DDF1C101F2370E020104
:1025D000026F00017FDDF0C101F2370E0201026FD0
:1025E000000178DDCBD10101F66B5B0EF56F0201C6
:1025F000016B370E026F00016DDD0A0E0201016FE3
:10260000370E026F000166DDF1C101F2370E0201E3
:10261000026F00015FDDF0C101F2370E0201026FAF
:10262000000158DDABD10101F66B5B0EF56F0201C5
:10263000016B370E026F00014DDD0B0E0201016FC1
:10264000370E026F000146DD0201016B370E026F8B
:10265000000140DD780E0201016F370E026F0001AC
:1026600039DD8CD10101F66B5B0EF56F0201016B58
:10267000370E026F00012EDD640E0201016F370E6E
:10268000026F000127DD7AD10101F66B5B0EF56F59
:10269000800E0201016F370E026F00011BDD020187
:1026A000016B370E026F000115DD68D10101F66B79
:1026B0005B0EF56F0201016B370E026F00010ADD40
:1026C000650E0201016F370E026F000103DD56D166
:1026D0000101F66B5B0EF56FFDC101F2370E0201D1
:1026E000026F0001F7DCFCC101F2370E0201026F3C
:1026F0000001F0DCEBC101F2370E0201026F0001B4
:10270000E9DCEAC101F2370E0201026F0001E2DCEE
:1027100035D10101F66B5B0EF56FFDC101F2370E8D
:102720000201026F0001D6DCFCC101F2370E02018A
:10273000026F0001CFDC22D10101F66B5B0EF56F59
:10274000FDC101F2370E0201026F0001C3DCFCC1C2
:1027500001F2370E0201026F0001BCDCE8C101F298
:10276000370E0201026F0001B5DC08D10101F66BE2
:102770005B0EF56FFDC101F2370E0201026F000121
:10278000A9DCFCC101F2370E0201026F0001A2DCDC
:10279000F5D00101F66B5B0EF56FFDC101F2370E4E
:1027A0000201026F000196DCFCC101F2370E02014A
:1027B000026F00018FDCEDC101F2370E0201026FE2
:1027C000000188DCECC101F2370E0201026F00014A
:1027D00081DCD4D00101F66B5B0EF56FFDC101F217
:1027E000370E0201026F000175DCFCC101F2370EE9
:1027F0000201026F00016EDCC1D00101F66B5B0EBD
:10280000F56FFDC101F2370E0201026F000162DCBB
:10281000FCC101F2370E0201026F00015BDCE9C16D
:1028200001F2370E0201026F000154DCA7D0010152
:10283000F66B5B0EF56FFDC101F2370E0201026F00
:10284000000148DCFCC101F2370E0201026F0001F9
:1028500041DC94D00101F66B5B0EF56FFDC101F216
:10286000370E0201026F000135DCFCC101F2370EA8
:102870000201026F00012EDCEEC101F2370E0201EF
:10288000026F000127DC7AD00101F66B5B0EF56F59
:10289000FDC101F2370E0201026F00011BDCFCC119
:1028A00001F2370E0201026F000114DC67D0010152
:1028B000F66B5B0EF56FFDC101F2370E0201026F80
:1028C000000108DCFCC101F2370E0201026F0001B9
:1028D00001DC54D00101F66B5B0EF56FFDC101F216
:1028E000370E0201026F00016AEC10F0FCC101F228
:1028F000370E0201026F00016AEC10F0320E020185
:10290000016F370E026F00016AEC10F037D0988625
:10291000000E86B6010E0201006F0101F66B5B0E20
:10292000F56FFDC101F2370E0201026F00016AEC82
:1029300010F0FCC101F2370E0201026F00016AECD7
:1029400010F000C201F2370E0201026F00016AECC2
:1029500010F014D00101F66B5B0EF56F0201016BF4
:10296000370E026F00016AEC10F0040E0201016FD5
:10297000370E026F00016AEC10F000D0000C01C2AB
:1029800003F200C202F203C203F0020102C2E9FF35
:1029900003C2EAFFEF5206E0022BD8B4032B00017A
:1029A000F2D702010051025D006E01510359036E1E
:1029B00000C001F0026E0001E7EF14F00101FF6BAF
:1029C000FE6B0201016B5B0E006F0001D8D702C0E5
:1029D00003F00150035205E101500101FE5D0DE2DB
:1029E0000001036A0101FE515B0FE96E000E032036
:1029F000EA6EEF50FF27FE2BE4D7FF1FFFC101F067
:102A0000000149EF15F0640E0201036F988086A063
:102A100004D0035302E00307F9D70251F2CF04F2C6
:102A2000F29E00014FEC00F0020104BFF28E956AA5
:102A30008C6E96908D9000D096908D800001000C49
:102A40000101FFBF11D00F0E006EFE3900160A0EF5
:102A5000005C03E2300E002602D0FF51002600C0C9
:102A600002F20001D0DF01010F0EFE170A0EFE5D1B
:102A700002E2300E02D0FF9FFF51FE27FEC102F29C
:102A80000001C1DF72EF15F00101FC6BFD6B00016D
:102A900095D701C0FDF1020E0201026F0001B3DF04
:102AA000036A0101FC515B0FE96E000E0320EA6E20
:102AB000EF5212E0036AFC515B0FE96E000E032037
:102AC000EA6EEFCFFEF1FEC102F200019CDF0101D0
:102AD000FC2B0001E5D70101FDC1FEF1370EFF6FB0
:102AE0000001AED7030E0201026F00018CDF000C63
:102AF000D56ACD6AB2EC0EF09D9AF29AF29CF29EE3
:102B0000F2BEFDD720EF17F094820A0E006E04008B
:102B1000002EFDD794800A0E006E0400002EFDD713
:102B20008B9294920A0E006E0400002EFDD78B90BB
:102B300094900101FE51FE0B0201016F0A6F00012A
:102B4000F7EC0CF002010A6B0001F7EC0CF0070E39
:102B50000101FF25E96E000E02010021EA6EEFCFB0
:102B600001F201C20AF20001F7EC0CF0060E0101BD
:102B7000FF25E96E000E02010021EA6EEFCF01F29F
:102B800001C20AF20001F7EC0CF0050E0101FF256D
:102B9000E96E000E02010021EA6EEF503F0B026F5A
:102BA0000A6F0001F7EC0CF0040E0101FF25E96E3D
:102BB000000E02010021EA6EEFCF01F201C20AF21B
:102BC0000001F7EC0CF0030E0101FF25E96E000E89
:102BD00002010021EA6EEFCF01F201C20AF2000108
:102BE000F7EC0CF0020E0101FF25E96E000E020168
:102BF0000021EA6EEFCF01F201C20AF20001F7EC08
:102C00000CF0010E0101FF25E96E000E020100210A
:102C1000EA6EEFCF01F201C20AF20001F7EC0CF00C
:102C200094920000948082A0FED70A0E006E0400E9
:102C3000002EFDD700D0000094820A0E006E040022
:102C4000002EFDD72DEF16F0D00E0101FE6FFDC155
:102C500000F2FCC1FFF1000157D771EF17F0F29CB1
:102C6000F29EF2BEFDD70201056B1C0E046F040E2E
:102C7000066F000159EC0FF001C0FBF100C0FAF142
:102C80000101FAC100F0FB51036E06E1020E005C87
:102C90000001D8B4AAD00101035006E1030E005C84
:102CA0000001D8B4ACD00101035006E1070E005C6E
:102CB0000001D8B4B5D00101035006E1640E005CF8
:102CC0000001D8B4C6D00101035006E1050E005C36
:102CD0000001D8B410D10101035006E1650E005C7B
:102CE0000001D8B412D10101035006E1060E005CC8
:102CF0000001D8B4F7D10101035006E1080E005CD1
:102D00000001D8B419D20101035006E1090E005C9C
:102D10000001D8B41BD20101035006E1660E005C2D
:102D20000001D8B432D20101035006E1670E005C05
:102D30000001D8B435D20101035006E1680E005CF1
:102D40000001D8B44ED20101035006E1690E005CC7
:102D50000001D8B451D20101035006E16A0E005CB3
:102D60000001D8B45FD20101035006E16B0E005C94
:102D70000001D8B462D20101035006E16C0E005C80
:102D80000001D8B47CD20101035006E16D0E005C55
:102D90000001D8B480D20101035006E16E0E005C40
:102DA0000001D8B48FD20101035006E16F0E005C20
:102DB0000001D8B493D20101035006E1700E005C0B
:102DC0000001D8B497D20101035006E1710E005CF6
:102DD0000001D8B4ADD20101035006E1720E005CCF
:102DE0000001D8B4B1D20101BCD20101FD6B020EC9
:102DF000FC6FFE6B00018DEC10F046DEBCD20101D1
:102E0000FD6B030EFC6FFE6B00018DEC10F03CDEE1
:102E1000640E0101FC6F00014BEC02F0FF00ABD22D
:102E2000F29CF29EF2BEFDD70101FD6B070EFC6F16
:102E3000FE6B00018DEC10F027DEB2EC0EF058D6E0
:102E4000640E0101FC6F00014BEC02F000EF5BF03F
:102E500092D20201056B200E046F020E066F000174
:102E600059EC0FF000C0E7F00201056B220E046F71
:102E7000020E066F000159EC0FF000C0E6F00201EF
:102E8000056B240E046F020E066F000159EC0FF063
:102E900000C0E5F00201056B260E046F020E066FFE
:102EA000000159EC0FF000C0E3F00201056B280EA1
:102EB000046F020E066F000159EC0FF000C0E2F043
:102EC0000201056B2A0E046F020E066F000159EC19
:102ED0000FF000C0E1F00101FD6BE00EFC6F00019E
:102EE000B3D60101FD6B640EFC6FFE6B00018DEC2F
:102EF00010F0CADD40D20101FD6B050EFC6FFE6BC8
:102F000000018DEC10F0C0DD36D2D8511508D8B0D4
:102F1000DFD00201056B200E046F040E066F000166
:102F200059EC0FF001C0EBF100C0EAF10201056BB2
:102F3000240E046F020E066F000159EC0FF000C062
:102F4000E8F10201056B260E046F040E066F000106
:102F500059EC0FF001C0EDF100C0ECF10201056B7E
:102F60002A0E046F020E066F000159EC0FF000C02C
:102F7000E9F10201056B2C0E046F040E066F0001CF
:102F800059EC0FF001C0EFF100C0EEF10101FC6B54
:102F9000EBC1FEF1EAC1FDF1000197EC0EF0020E6B
:102FA0000101FC6FEDC1FEF1ECC1FDF1000197ECF8
:102FB0000EF00101EEC100F0EF51036E05E1C80E05
:102FC000005C00012AE00101010E035C05E1900EA6
:102FD000005C000130E00101020E035C05E1580EC7
:102FE000005C000137E00101030E035C05E1200EE7
:102FF000005C00013EE00101030E035C05E1E80E08
:10300000005C000145E00101070E035C05E1D00E04
:10301000005C00014DE001015BD00101EF6BC80EC7
:10302000EE6F0001E96B3C0EE86FF70EEB6FDC0E04
:10303000EA6F01014DD0010E0101EF6F900EEE6FAE
:103040000001E96B780EE86FFB0EEB6FEE0EEA6F96
:1030500001013ED0020E0101EF6F580EEE6F00012C
:10306000E96BB40EE86FFD0EEB6F490EEA6F0101DC
:103070002FD0030E0101EF6F200EEE6F0001E96B00
:10308000F00EE86FFD0EEB6FF70EEA6F010120D036
:10309000030E0101EF6FE80EEE6F010E0001E96F04
:1030A0002C0EE86FFE0EEB6F5F0EEA6F010110D081
:1030B000070E0101EF6FD00EEE6F020E0001E96FF7
:1030C000580EE86FFF0EEB6F2F0EEA6F010100D074
:1030D0000101FD6B650EFC6FFE6B00018DEC10F0C5
:1030E000D3DC49D10201056B200E046F020E066F7E
:1030F000000159EC0FF0005206E1015204E10252C6
:1031000002E103520BE0010E0101E66FFD6BDA0EE6
:10311000FC6F000160EC02F0F28A03D00101E66B63
:10312000F29A0101FD6B060EFC6FE6C1FEF1000193
:103130008DEC10F0A9DC1FD10101FD6B080EFC6FB6
:10314000FE6B00018DEC10F09FDC15D10201056BC8
:10315000200E046F040E066F000159EC0FF001C041
:10316000FBF100C0FAF10101FA3D03D0FB3D01D0B3
:1031700004D0FBC1F1F1FAC1F0F1FD6B090EFC6F57
:10318000FE6B00018DEC10F07FDCFBC1FDF1FAC19C
:10319000FCF10101FE6B00018DEC10F075DCEBD051
:1031A0000201056B200E046F040E066F000159EC3E
:1031B0000FF001C0EBF100C0EAF10101FC6BEBC1C3
:1031C000FEF1EAC1FDF1000197EC0EF0FBC1FDF14B
:1031D000FAC1FCF10101FE6B00018DEC10F054DC32
:1031E000CAD0FBC1FDF1FAC1FCF10101FE6B000187
:1031F0008DEC10F049DCBFD00201056B200E046F8E
:10320000020E066F000159EC0FF000C0E8F1FBC19F
:10321000FDF1FAC1FCF10101FE6B00018DEC10F033
:1032200033DCA9D0FBC1FDF1FAC1FCF10101FE6B59
:1032300000018DEC10F028DC9ED00201056B200E01
:10324000046F040E066F000159EC0FF001C0EDF1A0
:1032500000C0ECF1020E0101FC6FEDC1FEF1ECC10A
:10326000FDF1000197EC0EF0FBC1FDF1FAC1FCF19C
:103270000101FE6B00018DEC10F006DC7CD0FBC17F
:10328000FDF1FAC1FCF10101FE6B00018DEC10F0C3
:1032900044EC15F070D00201056B200E046F020E95
:1032A000066F000159EC0FF000C0E9F1FBC1FDF120
:1032B000FAC1FCF10101FE6B00018DEC10F044EC51
:1032C00015F059D0FBC1FDF1FAC1FCF10101FE6B13
:1032D00000018DEC10F044EC15F04DD0FBC1FDF178
:1032E000FAC1FCF10101FE6B00018DEC10F044EC21
:1032F00015F041D00201056B200E046F020E066F1F
:10330000000159EC0FF000C0F4F10101F45303E0A7
:1033100098948F8402D098948F94FBC1FDF1FAC1E8
:10332000FCF1FE6B00018DEC10F044EC15F023D0A5
:10333000FBC1FDF1FAC1FCF10101FE6B00018DEC56
:1033400010F044EC15F017D0FBC1FDF1FAC1FCF10F
:103350000101FE6B00018DEC10F044EC15F00BD078
:103360000101FD6B010EFC6FFE6B00018DEC10F096
:1033700044EC15F000D0B2EC0EF0C00EF2123FEFAC
:103380001AF00101FE6BFD6BFC6BFD51FB5D1EE352
:1033900003E1FA51FC5D1AE25B0EFC25E96E000EBA
:1033A000FD21EA6EEFCF01F201C202F2000103EC4F
:1033B00015F05B0E0101FC25E96E000EFD21EA6EA1
:1033C000EF50FE27FC2BD8B4FD2BDFD7FE1FFE39B4
:1033D000006E0F0E00160050300FFF6FFE510F0BE6
:1033E000300F0201006F0101FF51390802E2070EA0
:1033F000FF2702010051390802E2070E0027FFC132
:1034000002F2000103EC15F000C202F203EC15F029
:10341000030E0201026F000103EC15F0000CF86AC4
:10342000D09E0D8EEA6AE96A7E86110EAF6E040E9A
:103430007F6EA60EAC6E900EAB6EC150C00B0F0926
:10344000C16E070EB46E196A1A6A010E0101F06F9F
:10345000F16BF26FF36BF56BF66B0001B5EF0EF0ED
:10346000988286B204D0F29CF29EF2BEFDD719EF8C
:1034700010F0C00EF212D7A102D02FEF16F001010A
:10348000E23D06D0E35304E1E45302E1E55350E0AA
:10349000E22D23D0E35321E1E4531FE1E5531DE185
:1034A000FD6B0B0EFC6FFE6B00018DEC10F044EC1D
:1034B00015F0EA6A5B0EE96EE26AF00EE16E780ED4
:1034C000016EE6CFEEFF012EFCD70101FB6B780EFB
:1034D000FA6F000156DF26D00101E251020823E114
:1034E000E35321E1E4531FE1E5531DE1FD6B0B0EB6
:1034F000FC6FFE6B00018DEC10F044EC15F0EA6AF5
:103500005B0EE96E010EE26E680EE16E780E016EE2
:10351000E6CFEEFF012EFCD70101FB6B780EFA6FB0
:1035200000012FDF0101E56BE46BE36BFF0EE26F3F
:10353000938081B008D0640EFC6F00014BEC02F068
:0C354000938081B000D000018BD7030005
:020000040030CA
:0E00000000260C1E838381000FC00FE00F400E
:00000001FF
